:100E2800000102030405060708090A0B0C0D0E0F42
:080E380041001000410011000F
:1009B80090E600E054E74410F000000090E604746C
:1009C80080F00000007406F0000000E4F000000071
:1009D80090E6107420F000000090E611F00000008E
:1009E80090E61274A2F000000090E61374A0F000E4
:1009F800000090E61474E2F000000090E61574E040
:100A0800F000000090E6047480F00000007404F028
:100A1800000000E4F000000090E6497482F0000055
:100A280000F000000090E6187410F000000090E656
:100A38001A740CF000000090E619E054FEF0000073
:100A48000090E61BE054FEF000000090E6917480F0
:100A5800F0000000F000000090E695F0000000F0C3
:070A680000000043AF012272
:1005A10078007C007D017BFF7A0E79287E007F1028
:1005B1001204FBC205E5AA30E2030206E2E5AA3015
:1005C100E7030206E275310075320490F400E0247D
:1005D100FE700302067524FA700302069124F87076
:1005E100030206BA240F60030206BE90FC007401E8
:1005F100F090F401E090FC01F090F402E090FC0234
:10060100F0D2B690F401E0701AA3E0701630B01386
:1006110074C0120D44C2B67F08120D4AD2B67F08CB
:10062100120D4A30B04690E694E0FE90E695E07CEB
:10063100002400FFEC3ECF24FCCF34FFFE7B017A87
:10064100F47904120AFB501C90FC0330B4117408B5
:10065100F07FE87E03120D4C7403120D44806A741E
:1006610004F0806590FC037402F0805D90FC0374DB
:1006710001F0805590FC007402F0E4A3F0A3F03087
:10068100B406A37410F0804190FC037420F080390B
:1006910075310075321190FC007408F07A007B000E
:1006A1007D017F50120D9E7F50120BCC7AFC7B0195
:1006B1007D107F50120D828010D202800C753100A6
:1006C10075320190FC0074AAF0E53190E69CF000CF
:1006D1000000E53290E69DF000000090E695748000
:0106E100F028
:0106E20022F5
:0C0D440090E601F07F147E007D007C0032
:100D50008F368E358D348C33783374FF120583ECE7
:060D60004D4E4F70F3221E
:0A0AFB008E338F348B358A3689372D
:100B0500E4F538F539C3E5399534E538953350338F
:100B1500AB35AA36A937853982853883120521FF79
:100B2500E4FEC2B2EF1392B7EFC313FFD2B20EBE0B
:100B350008F0C2B220B002C3220539E53970C605F6
:040B45003880C2D35F
:010B49002289
:02004100D322C8
:02004E00D322BB
:02005000D322B9
:080E460090E6BAE0F53BD3226F
:1007EB0090E740E53BF0E490E68AF090E68B04F06E
:0207FB00D32207
:080E4E0090E6BAE0F53AD32268
:100E160090E740E53AF0E490E68AF090E68B04F03D
:020E2600D322D5
:0207FD00D32205
:0208FB00D32206
:0208FD00D32204
:100CF70090E6B9E0242F600D04701990E604E0FF38
:100D0700430780800890E604E0FF53077F00000058
:070D1700EFF08002D322C3BC
:010D1E0022B2
:100DBA00C0E0C083C082D2015391EF90E65D740116
:080DCA00F0D082D083D0E032AA
:100DEA00C0E0C083C0825391EF90E65D7404F0D0F6
:060DFA0082D083D0E0323C
:100E0000C0E0C083C0825391EF90E65D7402F0D0E1
:060E100082D083D0E03225
:100C0400C0E0C083C08285130F85141085108285CF
:100C14000F83A37402F0850B11850C128512828553
:100C24001183A37407F05391EF90E65D7410F0D034
:060C340082D083D0E03203
:100DD200C0E0C083C082D2045391EF90E65D7408F4
:080DE200F0D082D083D0E03292
:1008BE00C0E0C083C08290E680E030E720850B0F59
:1008CE00850C10851082850F83A37402F085131199
:1008DE00851412851282851183A37407F05391EF4C
:0D08EE0090E65D7420F0D082D083D0E0321F
:01003200329B
:01004A003283
:01005200327B
:0107FF0032C7
:0108FF0032C6
:010E5E003261
:010E5F003260
:010E6000325F
:010E6100325E
:010E6200325D
:010E6300325C
:010E6400325B
:010E6500325A
:010E66003259
:010E67003258
:010E68003257
:010E69003256
:010E6A003255
:010E6B003254
:010E6C003253
:010E6D003252
:010E6E003251
:010E6F003250
:010E7000324F
:010E7100324E
:010E7200324D
:010E7300324C
:010E7400324B
:010E7500324A
:010E76003249
:010E77003248
:010E78003247
:010E79003246
:010E7A003245
:100B9000C0E0C083C08290E6D1E0900010F090E603
:100BA000D0E4F000000090E6D17402F000000053A1
:100BB00091BF00000090E66104F000000090E6990B
:0C0BC00004F075BB06D082D083D0E03278
:010E7B003244
:100D66001201000200000040E4E43211000001021A
:0C0D760000010001020203030404050553
:050E40000308FF0D6630
:10028D00E4F52CF52BF52AF529C204C200C203C2F0
:10029D0001C202D2B675B5C4D2B61209B8120E5645
:1002AD007E087F008E0D8F0E751508751612750B55
:1002BD0008750C1C75130875144A75170875187890
:1002CD00EE54C07003020398752D00752E808E2F8D
:1002DD008F30C374BC9FFF74089ECF2402CF3400AF
:1002ED00FEE48F288E27F526F525F524F523F52236
:1002FD00F521AF28AE27AD26AC25AB24AA23A92224
:10030D00A821C31205705031AE23AF24E5302FF56F
:10031D0082E52F3EF583E0FDE52E2FF582E52D3E9E
:10032D00F583EDF0EF2401F524E43EF523E43522C9
:10033D00F522E43521F52180B9852D0D852E0E741C
:10034D00002480FF740834FFFEC3E5169FF516E503
:10035D00159EF515C3E5109FF510E50F9EF50FC31E
:10036D00E5129FF512E5119EF511C3E50C9FF50CF5
:10037D00E50B9EF50BC3E5149FF514E5139EF513E0
:10038D00C3E5189FF518E5179EF517D2E843D82059
:10039D0090E668E0440BF090E65CE0443DF0000030
:1003AD0000E4F5A2000000D2AF90E680E020E10568
:1003BD00D20512000390E680E054F7F0538EF8C298
:1003CD00041205A130022190E680E054FDF0E054C6
:1003DD00F7F0750D0D750E66D20512000390E680CF
:1003ED00E04402F0C204C202300105120056C201FF
:1003FD003004CE12004150C9C204120D1F20001648
:10040D0090E682E030E704E020E1EF90E682E03014
:0E041D00E604E020E0E4120CA012004E80A3E2
:0B00360090E50DE030E402C322D3226D
:1000560090E6B9E0700302011514700302019224C0
:10006600FE700302021524FB700302010F147003D5
:100076000201091470030200FD1470030201032437
:10008600056003020279120050400302028590E6E1
:10009600BBE024FE602A14603B24FD601114602A34
:1000A60024067050E50D90E6B3F0E50E803C120094
:1000B60036503EE51590E6B3F0E516802D02027443
:1000C600E50F90E6B3F0E5108020E51190E6B3F079
:1000D600E512801690E6BAE0FF120CCCAA06A90734
:1000E600EA49600DEE90E6B3F0EF90E6B4F0020256
:1000F60085020274020274120E16020285120E4E58
:10010600020285120E460202851207EB02028512D2
:1001160007FD400302028590E6B8E0247F601514CF
:10012600601924027063A200E43325E0FFA203E411
:10013600334F8041E490E740F0803F90E6BCE054C6
:100146007EFF7E00E0D394807C0040047D01800227
:100156007D00EC4EFEED4F2478F582740D3EF5835E
:10016600E493FF3395E0FEEF24A1FFEE34E68F82A1
:10017600F583E0540190E740F0E4A3F090E68AF0BE
:1001860090E68B7402F00202850202741208FB40AC
:100196000302028590E6B8E024FE6016240260039E
:1001A60002028590E6BAE0B40105C20002028502A9
:1001B600027490E6BAE0705590E6BCE0547EFF7E8D
:1001C60000E0D394807C0040047D0180027D00EC39
:1001D6004EFEED4F2478F582740D3EF583E493FFD1
:1001E6003395E0FEEF24A1FFEE34E68F82F583E03F
:1001F60054FEF090E6BCE05480131313541FFFE046
:10020600540F2F90E683F0E04420F08072805F1256
:1002160008FD506B90E6B8E024FE60192402704E8B
:1002260090E6BAE0B40104D200805490E6BAE064E5
:1002360002604C803990E6BCE0547EFF7E00E0D33D
:1002460094807C0040047D0180027D00EC4EFEED32
:100256004F2478F582740D3EF583E493FF3395E0E1
:10026600FEEF24A1FFEE34E68F82F583800D90E643
:10027600A08008120CF7500790E6A0E04401F09029
:06028600E6A0E04480F058
:01028C00224F
:0300330002004682
:0400460053D8EF326A
:100CA00090E682E030E004E020E60B90E682E0305F
:100CB000E119E030E71590E680E04401F07F147E12
:0C0CC00000120B4A90E680E054FEF02287
:1000030030050990E680E0440AF0800790E680E03E
:100013004408F07FDC7E05120B4A90E65D74FFF026
:0F00230090E65FF05391EF90E680E054F7F02203
:080E5600E4F51ED2E9D2AF223F
:100BCC00AD0790E678E020E6F9C2E990E678E044DB
:100BDC0080F0ED25E090E679F090E678E030E0F9F1
:100BEC0090E678E04440F090E678E020E6F990E674
:080BFC0078E030E1D6D2E922D5
:100C6E00AC0790E678E020E6F9E51E702390E67872
:100C7E00E04480F0EC25E090E679F08D19AF03A901
:100C8E0007751A018A1B891CE4F51D751E01D322F6
:020C9E00C3226F
:100C3A00AC0790E678E020E6F9E51E702590E678A4
:100C4A00E04480F0EC25E0440190E679F08D19AF9C
:100C5A0003A907751A018A1B891CE4F51D751E0371
:040C6A00D322C322AC
:03004B000206E3C7
:1006E300C0E0C083C082C085C084C086758600C058
:1006F300D075D000C000C001C002C003C006C0074F
:1007030090E678E030E206751E060207CD90E678A3
:10071300E020E10CE51E64026006751E070207CDAA
:10072300E51E24FE605F14603624FE70030207BEDC
:1007330024FC70030207CA240860030207CDAB1A26
:10074300AA1BA91CAF1D051D8F82758300120521ED
:1007530090E679F0E51D65197070751E05806B9044
:10076300E679E0AB1AAA1BA91CAE1D8E8275830025
:1007730012054E751E02E5196401704E90E678E08D
:100783004420F08045E51924FEB51D0790E678E086
:100793004420F0E51914B51D0A90E678E04440F0D2
:1007A300751E0090E679E0AB1AAA1BA91CAE1D8E3C
:1007B3008275830012054E051D800F90E678E04494
:1007C30040F0751E008003751E005391DFD007D0E3
:1007D30006D003D002D001D000D0D0D086D084D0B0
:0807E30085D082D083D0E03202
:020CCC00A90776
:100CCE00AE17AF188F828E83A3E064037017AD0149
:100CDE0019ED7001228F828E83E07C002FFDEC3E99
:080CEE00FEAF0580DFE4FEFF0C
:010CF60022DB
:100D8200120C3AE51E24FA600E146006240770F372
:0C0D9200D322E4F51ED322E4F51ED32288
:100D9E00120C6EE51E24FA600E146006240770F322
:0C0DAE00D322E4F51ED322E4F51ED3226C
:100D1F0090E682E044C0F090E681F0438701000046
:040D2F00000000229E
:100B4A008E318F3290E600E054187012E53224019B
:100B5A00FFE43531C313F531EF13F532801590E612
:100B6A0000E05418FFBF100BE53225E0F532E531FD
:100B7A0033F531E5321532AE31700215314E60056A
:060B8A00120D3380EE2283
:100D33007400F58690FDA57C05A3E582458370F9D3
:010D4300228D
:100800001201000200000040E4E431110000010286
:1008100000010A06000200000040010009022E004B
:1008200001010080320904000004FF0000000705F8
:10083000020200020007050402000200070586020A
:100840000002000705880200020009022E000101D3
:100850000080320904000004FF00000007050202C6
:100860004000000705040240000007058602400022
:10087000000705880240000004030904180358001B
:100880006F00720063006F006D0020004C00740068
:1008900064002E0028035800500044002800420045
:1008A000610073006500640020006F006E0020008E
:0E08B000410058005500500050002900000083
:03004300020900AF
:030053000209009F
:10090000020DBA00020E0000020DEA00020DD20034
:10091000020C04000208BE000200320002004A007D
:10092000020052000207FF000208FF00020E5E00F4
:10093000020E5F00020E6000020E6100020E6200F5
:10094000020E630002004A00020E6400020E6500FF
:10095000020E6600020E6700020E6800020E6900B9
:10096000020E6A0002004A0002004A0002004A0029
:10097000020E6B00020E6C00020E6D00020E6E0085
:10098000020E6F00020E7000020E7100020E720065
:10099000020E7300020E7400020E7500020E760045
:1009A000020E7700020E7800020E7900020E7A0025
:0809B000020B9000020E7B0017
:03000000020A6F82
:0C0A6F00787FE4F6D8FD75813B020AB6E2
:10042B00E709F608DFFA8046E709F208DFFA803EB3
:10043B0088828C83E709F0A3DFFA8032E309F608A0
:10044B00DFFA8078E309F208DFFA807088828C8308
:10045B00E309F0A3DFFA806489828A83E0A3F608BC
:10046B00DFFA805889828A83E0A3F208DFFA804C96
:10047B0080D280FA80C680D4806980F2803380106D
:10048B0080A680EA809A80A880DA80E280CA8033D6
:10049B0089828A83ECFAE493A3C8C582C8CCC5834E
:1004AB00CCF0A3C8C582C8CCC583CCDFE9DEE7801E
:1004BB000D89828A83E493A3F608DFF9ECFAA9F09D
:1004CB00EDFB2289828A83ECFAE0A3C8C582C8CCF3
:1004DB00C583CCF0A3C8C582C8CCC583CCDFEADE0C
:1004EB00E880DB89828A83E493A3F208DFF980CC6E
:1004FB0088F0EF60010E4E60C388F0ED2402B40467
:10050B000050B9F582EB2402B4040050AF2323450D
:06051B00822390047B73B3
:10052100BB010CE58229F582E5833AF583E022508F
:1005310006E92582F8E622BBFE06E92582F8E222D9
:0D054100E58229F582E5833AF583E49322F3
:10054E00F8BB010DE58229F582E5833AF583E8F0E3
:10055E00225006E92582C8F622BBFE05E92582C88F
:02056E00F22277
:10057000EB9FF5F0EA9E42F0E99D42F0E89C45F0E1
:010580002258
:100581007401FF3395E0FEFDFC080808E6CF2FF665
:1005910018E6CE3EF618E6CD3DF618E6CC3CF6223E
:100A7B0002028DE493A3F8E493A34003F68001F202
:100A8B0008DFF48029E493A3F85407240CC8C3337C
:100A9B00C4540F4420C8834004F456800146F6DF4B
:100AAB00E4800B0102040810204080900E38E47E95
:100ABB00019360BCA3FF543F30E509541FFEE49340
:100ACB00A360010ECF54C025E060A840B8E493A307
:100ADB00FAE493A3F8E493A3C8C582C8CAC583CA32
:100AEB00F0A3C8C582C8CAC583CADFE9DEE780BEEA
:010E450000AC
:00000001FF
